:1043DE000000B30101010200000301FA0400FA0516
:1043EE0000020A0A5A0B000F0C00FA0D00030E0011
:1043FE00030F0132100096120132130AFA14010251
:10440E0015010217010A18010A1905321A010A1BB1
:10441E00010A1C053223011E2400642A00FA2B0017
:10442E00FA2C50782D003C2E00462F001E300064D2
:10443E003250783300003432FA3501643601643775
:10444E000150380A643C00643E003C3FFFFF40FFD1
:10445E00FF411450420A5A430AC8440532450078B7
:10446E004600FA47FFFF4802024C00FA4EFFFF508B
:10447E000404510596521432530B28540A965602D0
:10448E0002570546580002590A465A32FA5B010A8B
:10449E005C14325E000A5F00FE61FFFF64FFFF677F
:1044AE0001036A0A3C6B00006C3296780132790186
:1044BE0032FAFAFA0065006F00790083008D0097DA
:1044CE0000A100AC00B600C000CA00D400DE00E8B7
:1044DE0000F2005B0063006A0072007A00820089BD
:1044EE000091009900A100A800B000B800BF00C75D
:1044FE0000CF00D600DF00E600EE00F600400046DA
:10450E00004C00520059005F0065006B007100778F
:10451E00007D00830089008F0095009C00A200A8FA
:10452E0000AE00B400BA00C000C600CC00D200D964
:08453E0000DF00E500EB00F1D5
:10009E00AE32AF3374B48E048F05FF1200858C34EC
:1000AE008D35AE32AF3374B48E048F05FF12465FBA
:1000BE008C328D33E5334532601374B4C39533FF00
:1000CE00E49532FE8E328F3378341246ABE551A86A
:1000DE0034B80015D395354010E551C39535FFE47E
:1000EE009534FE8E348F358010E5512402C395353C
:1000FE00FFE49534FE8E348F3522900073E0B40108
:10010E0004C20B8002D20B900074E0B40104C20C46
:10011E008002D20C9000B1E075F069A4FFAEF074CD
:10012E000A8E048F05FF120085900799ECF0A3ED5F
:10013E00F0A208401674038C068D07124644740113
:10014E00124636900797EEF0A3EFF07E017F0090F7
:10015E00006FE01246449000B2E08E048F05FF124D
:10016E000085740AFF1200858D3A9000BBE075F091
:10017E0069A4FFAEF0740A8E048F05FF12008590FD
:10018E00079DECF0A3EDF09000BDE060139000BD74
:10019E00E0F5F0741684FF7E00EF9007A5F0800660
:1001AE0074649007A5F090009CE0B40B0874E39083
:1001BE00005EF0804990009CE0B419129000B2E00D
:1001CE009044AD124627E49390005EF0803090008C
:1001DE009CE0B41E129000B2E09044CB124627E48D
:1001EE009390005EF0801790009CE0B42810900071
:1001FE00B2E09044F5124627E49390005EF0900032
:10020E00CFE0B40117900020740FF0A374FFF090AC
:10021E000022E4F0A3F074029000CFF09000CFE043
:10022E00B40341900022E0FEA3E0FF900020E0FC2A
:10023E00A3E0FD1246A3741012464474081246360B
:10024E00EF90005BF0EF700674FF90005BF07400AF
:10025E009000CFF0900021E090005CF0900020E044
:10026E0090005DF022C293C294C291C292C287C224
:10027E0090E5B554EFF5B5E5B554DFF5B5C296C2C8
:10028E0095C2A0C297C2A2C2A1E5B5547FF5B5E54D
:10029E00B554BFF5B5E5B554FBF5B5C20D7536468B
:1002AE007537467538009000A9E07005754A0280D2
:1002BE0003754A0390000874FFF0A374DCF09000FD
:1002CE008AE090000EF8E4F0E8A3F0C212C21474B3
:1002DE00C8900024F074C8900026F075250075248F
:1002EE0000C208756D00E54CB40903754C00753DF0
:1002FE0000900016E4F0A3F0754D1E7527007526CC
:10030E0000C210C211900799E0FEA3E0FF74031221
:10031E0046447401124636900797EEF0A3EFF0C2F2
:10032E000390000CE4F0A3F0C21B22053E2285A729
:10033E005075A7109000A7E0B4031EA2D8B34002D8
:10034E00C293A2D9B34002C294A2DAB34002C291C0
:10035E00A2DBB34002C2928012A2D8B34004C29371
:10036E00C291A2D9B34004C294C292A2DCB340029D
:10037E00C287A2DDB34002C29075D8408550A72235
:10038E00900047E4936406600280FE74C890079F55
:10039E00F8E4F0E8A3F075B50075840175A7007553
:1003AE00FF8075EF0690002EE4F075C91075A70F4B
:1003BE0075A1C775A70075D90075CE0C75A70F75F9
:1003CE00F1FE75F2FF75F30775F47875A4BA75A58D
:1003DE00FF75A60775AE0075AFFF75D48175D5FF95
:1003EE0075D6FF75D7FF75A70075A20175A1477564
:1003FE00F80975D80075D90475A71075D80075D988
:10040E000475DA0975DB0975DC0975DD0975DE0918
:10041E0075DF0975D84075A70075E60875E7107584
:10042E00BC0175BE0475BD6C75BE0775BDA075BEED
:10043E000875BD0175BC0075BB1875BC2075BA0872
:10044E0075E88075D11375A70F75E10575E2007516
:10045E00C740C293C294C291C292C287C290E5B500
:10046E0054EFF5B5E5B554DFF5B5C296C295C2A009
:10047E00C297C2A2C2A1E5B5547FF5B5E5B554BF8A
:10048E00F5B5E5B554FBF5B5759700759780740A0B
:10049E001200757597C0E5975420700280F8758F1D
:1004AE000275A700D2AF75980075A90C75A70F75C8
:1004BE00AB4375ADFB75AC1E75A71075C91875CA23
:1004CE000075CB0075C80475A700758912758E046A
:1004DE00758C00758A00C2A9D28C758D00758B0043
:1004EE00D2ABD28E75D944753100753000752D00A2
:1004FE00752C00754700754800C29974C8F50975CA
:10050E0008001226CA75B500746390079FF8E4F0D0
:10051E00E8A3F01229567464F5097508001226CA6C
:10052E00C21A900049E0B40108A2B54002D21A8066
:10053E002E900049E0B4021175A70F75F30F75A741
:10054E0000A2A34002D21A8016900049E0B4030F15
:10055E0075A70F75F31775A700A2A44002D21AA2B1
:10056E001AB3500302065B740890079FF8E4F0E894
:10057E00A3F01228257464F5097508001226CA74B2
:10058E000990079FF8E4F0E8A3F01228257464F5AB
:10059E00097508001226CA740A90079FF8E4F0E85D
:1005AE00A3F01228257464F5097508001226CA7482
:1005BE000B90079FF8E4F0E8A3F01228257464F579
:1005CE00097508001226CA740C90079FF8E4F0E82B
:1005DE00A3F01228257464F5097508001226CA7452
:1005EE000D90079FF8E4F0E8A3F01228257464F547
:1005FE00097508001226CA740E90079FF8E4F0E8F9
:10060E00A3F01228257464F5097508001226CA7421
:10061E00029000A8F0900049E090006CF090004924
:10062E00E0B401087400900074F0801C900049E062
:10063E00B4020874009000B7F0800D900049E0B449
:10064E00030674009000C4F0D21702073B90079F78
:10065E00E4F0A304F01228257464F509750800125D
:10066E0026CA740290079FF8E4F0E8A3F01228253A
:10067E007464F5097508001226CA740390079FF872
:10068E00E4F0E8A3F01228257464F5097508001249
:10069E0026CA740490079FF8E4F0E8A3F012282508
:1006AE007464F5097508001226CA740590079FF840
:1006BE00E4F0E8A3F01228257464F5097508001219
:1006CE0026CA740690079FF8E4F0E8A3F0122825D6
:1006DE007464F5097508001226CA740790079FF80E
:1006EE00E4F0E8A3F01228257464F50975080012E9
:1006FE0026CA74019000A8F0900049E090006CF0BA
:10070E00900049E0B401087400900074F0801C90D1
:10071E000049E0B4020874009000B7F0800D90001C
:10072E0049E0B4030674009000C4F0C217122ACA3E
:10073E009000B2E07006740A9000B2F090005EE095
:10074E00700674E390005EF0120108E5B54401F501
:10075E00B57406900038F07401900039F07403906F
:10076E00003BF0740490003CF0742C90003DF0744B
:10077E000590003EF0740390003FF074009000442A
:10078E00F07400900045F07401900046F0740090F3
:10079E000047F074FF900048F07453900136F074E7
:1007AE0075900137F07462900138F07461900139E0
:1007BE00F0747290013AF0747590013BF0742090D1
:1007CE00013CF0743490013DF0744390013EF0749E
:1007DE007990013FF0746C900140F07420900141CB
:1007EE00F07436900142F0742B900143F074379000
:1007FE000144F09000CEE090005BF0900085E09018
:10080E00005CF0900086E090005DF0C212C214749D
:10081E00C8900024F074C8900026F0C210C211A235
:10082E00B6B39209A2B3B3920A752500752400756A
:10083E003646753746753800754D1E900057E4F0F4
:10084E0075261975276490000874FFF0A374DCF008
:10085E00C20D754C00C20875290075280090000C59
:10086E00E4F0A3F0743A90075FF074FD900760F027
:10087E00756E00900058E4F0752B00752A009000FC
:10088E0010E4F0A3F090008AE090000EF8E4F0E897
:10089E00A3F090006BE075F032A4FFAEF090001E56
:1008AE00EEF0A3EFF0900799E0FEA3E0FF740312C1
:1008BE0046447401124636900797EEF0A3EFF0759A
:1008CE004B0174FA900034F0C21B756D00753D003B
:1008DE00C20EC20FC21CC203754E00C204D205C2A4
:1008EE0006D207C218C219753900754500753B004E
:1008FE00753F32754000754100743C900032F075C2
:10090E004200743C900033F0754300754400900033
:10091E0016E4F0A3F0754600D2B2D2A4D2B0D2B192
:10092E00D2A3D2A7D2A6D2A5D2B790006BE0D39411
:10093E00FA400674FA90006BF07E017F0090005D25
:10094E00E012464490005CE02FFF50010E90002014
:10095E00EEF0A3EFF0EFD394FFEE940F400790006C
:10096E0020E4F0A3F090005BE0700674FF90005B53
:10097E00F09000A8E0D39402400674019000A8F015
:10098E009000A9E07005754A028003754A03900035
:10099E00AAE0D39401400674009000AAF09000B033
:1009AE00E0C3940A5006740A9000B0F09000BAE0CA
:1009BE00700674019000BAF09000BAE0B4FF0674AD
:1009CE00FE9000BAF09000C1E0D394FE400674FE93
:1009DE009000C1F074019000C7F074019000C8F04F
:1009EE0074009000CAF074009000CFF0D29CD2EC4C
:1009FE0075CF01A298B35003020DF4C298E5486476
:100A0E00046006E59964FF6002801EE54860087484
:100A1E00E62548900034F0754800E547600874F00C
:100A2E002547900034F0754700E5486003020AD967
:100A3E00754800E599B4FF03754701E599B4FE03C7
:100A4E00754702E599B4FD03754703E599B4FC03B8
:100A5E00754704E599B4FA03754705E599B4FB03A8
:100A6E00754801E599B4F903754804E599D394E501
:100A7E004007E599C394F040028016859949754860
:100A8E00027E017F00E549C394E61246448E2E8F06
:100A9E002F753100753000E599D394C74007E5995D
:100AAE00C394E64002801F85994975480374E5C3D7
:100ABE009549F52F752E00AE2EAF2F904274120071
:100ACE00647830124689D299020DF4E548B40102D9
:100ADE008003020BB7E53145307003120273AE305E
:100AEE00AF3190005F12466BE599F078301246AB4D
:100AFE00AE30AF31EFB40106EEB407028003020B45
:100B0E00B790075FE0B43C028003020BA1C29C12B7
:100B1E00010890005BE09000CEF090005CE0900049
:100B2E0085F090005DE0900086F0A217403275517E
:100B3E0001E551D394075026E55190079FF8E4F054
:100B4E00E8A3F074AA90002EF01226F67464F5094C
:100B5E007508001226CA7851740126F650D38030DB
:100B6E00755108E551D3940E5026E55190079FF824
:100B7E00E4F0E8A3F074AA90002EF01226F6746446
:100B8E00F5097508001226CA7851740126F650D35D
:100B9E00122ACA74C890079FF8E4F0E8A3F0D29C1A
:100BAE007548007547007599FBE548B4020280034D
:100BBE00020C4BE5314530700685992D752C00AE33
:100BCE0030AF3174016F4E701BAC2CAD2DAA2EAB15
:100BDE002FED2BFBEC3AFA8A068B0790005F12463C
:100BEE006BE599F078301246ABAE30AF3174026FD0
:100BFE004E704AAC2CAD2D740D6D4C7027746390F5
:100C0E00079FF8E4F0E8A3F074AB90002EF090008C
:100C1E006CE0900049F0122A2F74C890079FF8E4F8
:100C2E00F0E8A3F0AE2CAF2D74566F4E7003120287
:100C3E0073120108854999754800754700E548B457
:100C4E00033FAE30AF3190005F12466BE599F078FE
:100C5E00301246ABAE30AF31AC2EAD2F8F028E03BD
:100C6E008C068D079042B0120064E493F9740193E0
:100C7E00FEEAD39EEB994009854999754800754760
:100C8E0000E548B404028003020DF4E531453070EE
:100C9E0003120273AE30AF3190005F12466BE599CE
:100CAE00F078301246ABAE30AF31EFB40006EEB492
:100CBE0001028003020DF4900042E075F002A4FDE3
:100CCE00ACF08D51ED90005F124680EDFAE0FBEA3C
:100CDE00900062124680EBFAE0FBEA2BFA9000429B
:100CEE00E0B502028003020DE50DED90005F1246A5
:100CFE0080E551FDE0FAED900063124680EAFDE0DA
:100D0E00FAEDC39AFD900042E0B505028003020D94
:100D1E00E5E551900061124680E551FDE0FAED9057
:100D2E000064124680EAFDE0FAED2AFD900042E0F2
:100D3E00B505028003020DE5E5519000651246806F
:100D4E00FDE0FAED900042E0F4042A900049F0E54F
:100D5E0051900066124680FDE0FAED900042E0F4FC
:100D6E00042A90004AF0E551900067124680FDE09B
:100D7E00FAED900042E0F4042A90004BF0E5519019
:100D8E000068124680FDE0FAED900042E0F4042A7D
:100D9E0090079FF8E4F0E8A3F074AB90002EF012E9
:100DAE002A2F7464F5097508001226CA90079F123F
:100DBE004652122A2F7464F5097508001226CA903D
:100DCE00079F124652122A2F7599F97464F5097508
:100DDE0008001226CA80FE7599FF7464F50975081D
:100DEE00001226CA80FEE5476006A299B3B34003FF
:100DFE00020F55C299E547B4011FAE30AF319000D6
:100E0E003812466BE0F59978301246ABAE30AF3102
:100E1E0074116F4E7003754700E547B40203854B9E
:100E2E0099E547B4031DAE30AF3190005F12466BAB
:100E3E00E0F599EFB40107EEB4070375470078307B
:100E4E001246ABE547B404028003020F34E5314588
:100E5E00307003852599AE30AF3174016F4E70033B
:100E6E00853999AE30AF3174026F4E7003853B9960
:100E7E00AE30AF3174036F4E7003853F99AE30AF15
:100E8E003174046F4E7003854199AE30AF317405E5
:100E9E006F4E7003854299AE30AF3174066F4E704F
:100EAE0003854399AE30AF3174076F4E700385449E
:100EBE0099AE30AF3174086F4E7006900017E0F5A2
:100ECE0099AE30AF3174096F4E7006900034E0F574
:100EDE0099AE30AF31740A6F4E7003854599AE30BE
:100EEE00AF31740B6F4E7003854099AE30AF3174D5
:100EFE000C6F4E7003854699AE30AF31740D6F4E48
:100F0E007005900034E4F0AE30AF31740D6F4E705A
:100F1E00037599FC78301246ABAE30AF31740E6F5C
:100F2E004E7003754700E547B4051CAE30AF3190E7
:100F3E0043DE12466BE493F59974E36F4E700375BE
:100F4E00470078301246ABE54864016005E548B4C9
:100F5E0004030209FEC28E7E087F00E53E1246445F
:100F6E00E58D75F008A4FDACF0EF2DFDEE3CFCE533
:100F7E008B75F02084FF7E00ED2FFFEC3EFE8E265B
:100F8E008F27D28E90008CE0605690001812465239
:100F9E00900018E0FCA3E0FD90001AE0FAA3E0FB3D
:100FAE00EDB5033CECB50238B216A208B34013A25D
:100FBE0016B34008E5B54404F5B58006E5B554FB17
:100FCE00F5B590001AE0FEA3E0FF90001CE0FCA334
:100FDE00E0FDEF2DFDEE3CFC90001AECF0A3EDF0E1
:100FEE00900099E06009900099E0C394034002805C
:100FFE006F123FCAA208B35009900057E0C394087D
:10100E0040028006900083E0F56CE56C75F005A457
:10101E00FFAEF09007A1EEF0A3EFF0900070E0C3EA
:10102E00953B4007E539C3953A50079007A1E4F088
:10103E00A3F0AE59AF5A9007A1E0FCA3E0FDEFD3A9
:10104E009DEE9C4004C2A1800B900057E0C3940C0F
:10105E005002D2A1900099E0B40205A2A1B392A2CF
:10106E00900099E0B4031C1240C6AE59AF5A9007D7
:10107E00A1E0FCA3E0FDEFD39DEE9C4004D2A18045
:10108E0002C2A1900074E06009A2B3300A01B3B3AA
:10109E0040028055A2B3300A01B3404DA2B3300CCA
:1010AE0001B340389000A7E0B40306A218B3B340D2
:1010BE000280067405900034F0D218A20DB34004DD
:1010CE0005388013C28E758D00758B00753E0075C8
:1010DE002701752600D28EA20CB3920AA20CB33051
:1010EE00B301B34004A20C920AA2B6300901B35068
:1010FE0003021535A2B6300901B35003021535A20D
:10110E00B6300B01B3500302142E754B000537E5B4
:10111E0038B40105753701800EE53864026005E5C7
:10112E0038B40303753704E538D3940340067404CA
:10113E00900034F0E53764046005E537B40704E544
:10114E0038600280067402900034F0753800E5377E
:10115E006401600AE537B404028003021429E537FE
:10116E00B401057536028003753601754A0190008B
:10117E008CE07013A20BB34008E5B554FBF5B580B7
:10118E0006E5B54404F5B5E536B4024990008CE0A9
:10119E006043900018E0FEA3E0FF90008CE08E0408
:1011AE008F05FF12008574018C068D07124636904E
:1011BE00001CEEF0A3EFF090001CE0F8A3E090000E
:1011CE001AC8F0A3C8F0900018E4F0A3F0C216E518
:1011DE00B554FBF5B5AE2AAF2BAC26AD27EF2DFDE2
:1011EE00EE3CFC8C2A8D2BAE26AF27EFD39DEE9CCA
:1011FE004011900010E0FAA3E0FBEBC394E8EA94F0
:10120E000340028006900010124652900008E52618
:10121E00F0A3E527F090000AE526F0A3E527F0AE4F
:10122E0026AF2774128E048F05FF1200858C288D31
:10123E0029C28E758D00758B00753E007527017560
:10124E002600D28E900008E0FEA3E0FFEF4E600B6A
:10125E007C7F7DCB1245468E248F25AE24AF257420
:10126E0028BE00039F5010E53D2FFF50010E740164
:10127E001246368E248F2585253D9000B0E0A82499
:10128E00B8000DD395254008E525900031F0800972
:10129E009000B0E014900031F0123D0C9000A7E0E9
:1012AE00B4030890002AE0653660028026A218B3C7
:1012BE004004D2198002B219900074E0600BA2189B
:1012CE00B35006A219B3B3400280067404900034E2
:1012DE00F0C218E54CB40903754C00A20E5003027F
:1012EE0013C6900065E0B4015AE54175F00584FF20
:1012FE007E0090055F12466BE0F533753200AE321C
:10130E00AF33900063E012464474648E048F05FF81
:10131E0012008574C18C068D071246448E348F35AB
:10132E0090000EE0FEA3E0FFAC32AD33120003746A
:10133E00648E048F05FF12008590000EECF0A3ED75
:10134E00F0800F900063E075F0C1A4FFAEF08E3414
:10135E008F35E53BC394CC505D75A71085F951854B
:10136E00FA527E017F00E552124644E5512FFF509E
:10137E00010E8E328F33AC34AD35EF2DFDEE3CFCCD
:10138E008C348D35D293D294E535F5FBE534F5FCEE
:10139E00E535F5E9E534F5EA9000A7E0B40314D29B
:1013AE0091D292E535F5EBE534F5ECE535F5EDE565
:1013BE0034F5EE75A700D20EE54AB40103754A0066
:1013CE009000ACE0D39401400D9000B3E0A824B897
:1013DE0000069525400280169000ACE0B40305751A
:1013EE004D038002C2007409900034F08019754DCF
:1013FE0001E536B401069000377401F0E536B4020B
:10140E00067402900037F0900008E0FEA3E0FFEFB4
:10141E00D39400EE947D4003120273A20BB3920993
:10142E00A20BB330B601B35003021535754B0190C4
:10143E00008CE07013A20BB34008E5B54404F5B57B
:10144E008006E5B554FBF5B5A20B9209E537D394AA
:10145E00484012D20DE537D3944B400974059000E5
:10146E0034F0753746A20D4013C28E758D00758B04
:10147E0000753E00752701752600D28EE54A60067E
:10148E00E5B54401F5B59000B4E0B40107E544C3F9
:10149E009414400280031202737408900057F0A255
:1014AE0004300501B35017A204B34008E5B5440853
:1014BE00F5B58006E5B554F7F5B5A2049205A2067A
:1014CE00300701B35017A206B34008E5B54402F544
:1014DE00B58006E5B554FDF5B5A2069207E544C301
:1014EE0094415009740E900034F012027390003E35
:1014FE00E0FE90003AE0C39E400990003AE0D3949B
:10150E0006400974FB900034F0120273900043E021
:10151E006015900043E0FE90003DE06E600974FEA1
:10152E00900034F0120273A210B3B35006E5376484
:10153E00016003021611A202B35006A200B3B3401B
:10154E000302160D75A71085F95185FA527E017F9B
:10155E0000E552124644E5512FFF50010E8E328F98
:10156E0033900014E0FCA3E0FDEF2DFDEE3CFC8C6F
:10157E00348D359000A7E0B4034EA208B34028A2E4
:10158E0019B3400CE535F5FBE534F5FCD293800A32
:10159E00E535F5EBE534F5ECD291A203B34004D278
:1015AE00A08002C2A0801FE535F5FBE534F5FCE511
:1015BE0035F5EBE534F5ECD293D291A203B34004AA
:1015CE00D2A08002C2A08011E535F5FBE534F5FC12
:1015DE00D293A203B34002D2919000C5E0B4021C94
:1015EE00AE32AF33AC57AD58EF2DFDEE3CFC8C3424
:1015FE008D35E535F5FDE534F5FED28775A700C2CC
:10160E0010D211A211B3B35006E537640460030281
:10161E0016EDA202B35006A200B3B340030216E9C0
:10162E0075A71085F95185FA527E017F00E5521299
:10163E004644E5512FFF50010E8E328F3390001429
:10164E00E0FCA3E0FDEF2DFDEE3CFC8C348D3590DF
:10165E0000A7E0B4034EA208B34028A219B3400C71
:10166E00E535F5E9E534F5EAD294800AE535F5ED90
:10167E00E534F5EED292A203B34004D2A08002C2AA
:10168E00A0801FE535F5E9E534F5EAE535F5EDE53C
:10169E0034F5EED294D292A203B34004D2A08002CB
:1016AE00C2A08011E535F5E9E534F5EAD294A2033E
:1016BE00B34002D2929000C5E0B4021CAE32AF33FA
:1016CE00AC57AD58EF2DFDEE3CFC8C348D35E53529
:1016DE00F5CEE534F5CFD29075A700D210C211E544
:1016EE004DB4081612363BA210B35005A211B340EA
:1016FE00028004D210D211754D1EE54DB4070612AC
:10170E0033F3754D08E54DB4063D90000EE0FEA393
:10171E00E0FFEF4E6006A208B3B340028023AE5343
:10172E00AF5490000EE0FCA3E0FDEF2DFDEE3CFC6F
:10173E008C538D54E536D39401500690000E120052
:10174E00391231C5754D07E54DB4050612302575B4
:10175E004D06E54DB4043290009AE09026ACF82880
:10176E002873122CB98012122CB9800D122E67809C
:09177E0008122F198003122F1923
:0F26AC0002177002177502177A02177F02178440
:1017870090007CE06005123DF58002C204754D05AE
:10179700E54DB40302800302188190007FE06005E5
:1017A700123EE58002C20690009AE0D39402403FC1
:1017B70090006EE02403A824B800049525500990F2
:1017C7000070E0D3953B50028008D2027408900065
:1017D70034F090006EE0A824B80005D39525500B8F
:1017E700900070E02403C3953B5002C202803990F9
:1017F700006EE02403A824B8000495255007E539B6
:10180700C3953A40028008D2027408900034F090E1
:10181700006EE0A824B80005D395255009E53A24C1
:101827000FC395395002C2029000B4E07007E54437
:10183700C3941440028002D202A2024005754D04EF
:10184700800A754D1E900016E4F0A3F0A208B3407D
:1018570029E54175F00584FF7E0090055F12466B10
:10186700E0C394695005123D41800F900799E0F855
:10187700A3E0900797C8F0A3C8F0E54DB40A5490C9
:101887000025E0C394465008C2967446900025F0A0
:10189700855B3375320075510112009EE535900066
:1018A70025F0900004E532F0A3E533F0C21390076A
:1018B7009BE0F532A3E0F53375510112009EE53543
:1018C700900024F0900000E532F0A3E533F0C21257
:1018D700754D03900024E0B536028003021972A209
:1018E70012406B900000E0FEA3E0FFEF4E605DAC9E
:1018F70024AD25740ABC0033D39D402FAA28AB29F9
:1019070074058A048B05FF1200858D068C079000ED
:1019170000E0FCA3E0FDCFCECF1200037401124616
:1019270036900000EEF0A3EFF08021AE28AF2990AB
:101937000000E0FCA3E0FD120003740A8E048F058B
:10194700FF120085900000ECF0A3EDF0D212AE2656
:10195700AF27900000E0FCA3E0FDEFC39DEE9C40A5
:101967000AD296C21274C8900024F0A212B3B350E0
:1019770007900024E0B53602800AD29674C890001A
:1019870024F0C212900025E0B536028003021A2324
:10199700A213406B900004E0FEA3E0FFEF4E605DF2
:1019A700AC24AD25740ABC0033D39D402FAA28ABC5
:1019B7002974058A048B05FF1200858D068C079014
:1019C7000004E0FCA3E0FDCFCECF120003740112A8
:1019D7004636900004EEF0A3EFF08021AE28AF2941
:1019E700900004E0FCA3E0FD120003740A8E048F4C
:1019F70005FF120085900004ECF0A3EDF0D213AEC2
:101A070026AF27900004E0FCA3E0FDEFC39DEE9C0A
:101A1700400AC2967446900025F0C213A213B3B3CE
:101A27005007900025E0B53602800AC296744690AA
:101A37000025F0C213E54DB40B5F900027E0C39477
:101A47004650139000B5E0B40104C2968002C295D7
:101A57007446900027F0855B33753200755102128A
:101A6700009EE535900027F0900006E532F0A3E5EB
:101A770033F0C21590079BE0F532A3E0F5337551BB
:101A87000212009EE535900026F0900002E532F044
:101A9700A3E533F0C214754D03900026E0B5360276
:101AA7008003021B43A214406B900002E0FEA3E0F8
:101AB700FFEF4E605DAC24AD25740ABC0033D39DA7
:101AC700402FAA28AB2974058A048B05FF120085CD
:101AD7008D068C07900002E0FCA3E0FDCFCECF126D
:101AE70000037401124636900002EEF0A3EFF08077
:101AF70021AE28AF29900002E0FCA3E0FD1200030D
:101B0700740A8E048F05FF120085900002ECF0A383
:101B1700EDF0D214AE26AF27900002E0FCA3E0FD63
:101B2700EFC39DEE9C40159000B5E0B40104D2963A
:101B37008002D295C21474C8900026F0A214B3B3E1
:101B47005007900026E0B5360280159000B5E0B446
:101B57000104D2968002D29574C8900026F0C21470
:101B6700900027E0B536028003021C0AA215406BDD
:101B7700900006E0FEA3E0FFEF4E605DAC24AD25CC
:101B8700740ABC0033D39D402FAA28AB2974058A59
:101B9700048B05FF1200858D068C07900006E0FC7C
:101BA700A3E0FDCFCECF120003740112463690009A
:101BB70006EEF0A3EFF08021AE28AF29900006E0F3
:101BC700FCA3E0FD120003740A8E048F05FF1200C8
:101BD70085900006ECF0A3EDF0D215AE26AF279066
:101BE7000006E0FCA3E0FDEFC39DEE9C40159000CE
:101BF700B5E0B40104C2968002C2957446900027EE
:101C0700F0C215A215B3B35007900027E0B536020E
:101C170080159000B5E0B40104C2968002C29574A5
:101C270046900027F0C215E54DB4027E123AA41281
:101C37003BBB90005FE02546F55B900797E0FEA36E
:101C4700E0FF740A12464490000AE0FCA3E0FD742A
:101C5700128F02FF1200858D078C038E048A058B75
:101C67000612454690079BEEF0A3EFF074F0BE0016
:101C7700039F500B74F090079BF8E4F0E8A3F090F3
:101C8700079BE0FEA3E0FFE55B2FFF50010E9007E7
:101C97009BEEF0A3EFF0900037E0B40103754D0A17
:101CA700900037E0B40203754D0BE54DB401259064
:101CB70000CCE09026BBF828287312384280121215
:101CC7003842800D1238CC800812397880031239D7
:011CD7007894
:0F26BB00021CC1021CC6021CCB021CD0021CD583
:101CD800754D029000B7E0B402028003021DF39034
:101CE800005AE0D39540506490005AE0F40425402F
:101CF800FE9000BAE08E00F5F0E884FF7E008F5178
:101D0800EFC39410500CEF8551F0A4FDACF08D5149
:101D180080037551FF90005AE0D39551400B900015
:101D28005AE0C39551F54E8003754E009000D5E0FA
:101D3800D3954E40069000D5E0F54E9000D6E0C30E
:101D4800954E50069000D6E0F54E807190005AE00E
:101D5800C39540FE9000BAE08E00F5F0E884FF7E5F
:101D6800008F51EFC39410500CEF8551F0A4FDACD7
:101D7800F08D5180037551FF855133753200900005
:101D88005AE02533FFAE3250010E8E328F3374FF86
:101D9800BE0009D39F400585334E8003754EFF90E2
:101DA80000D5E0D3954E40069000D5E0F54E900062
:101DB800D6E0C3954E50069000D6E0F54EA208B383
:101DC800B350099000C2E0D3954F5002800A7407BF
:101DD800900034F0C297801375A710E5CDC3954ED7
:101DE8004004C2978002D29775A700E54CC39409B6
:101DF8004003022448A2EDB35003022448C2EDE593
:101E08004C6003021EC6900068E07003021EB57E97
:101E1800017F00E5BE124644E5BD2FFF50010E8E3E
:101E2800328F33900068E0B4011874101246449061
:101E3800005EE08E048F05FF120085ED900030F003
:101E4800802CAE32AF33741012464490005EE08EA0
:101E5800048F05FF120085900030E02DFD50010C25
:101E680074018C068D07124636EF900030F0E54578
:101E780060089000C4E06402600280219000C6E01F
:101E8800B4011A900030E075F0E7A4FFAEF0E54524
:101E98008E048F05FF120085ED900030F090009AB7
:101EA800E064016006900030E0F539800375390080
:101EB800900064E07005754C01800375BB18E54C13
:101EC800B40102800302205E900064E070030220E7
:101ED8004D7E017F00E5BE124644E5BD2FFF50014F
:101EE8000E8E328F339000AAE0B4010F7E0F7FFF71
:101EF800AC32AD331246A38E328F339000CFE0B4AC
:101F08000245AE32AF33900020E0FCA3E0FDEDD3F4
:101F18009FEC9E400A900020E532F0A3E533F0AE36
:101F280032AF33900022E0FCA3E0FDEFD39DEE9C9E
:101F3800400A900022E532F0A3E533F0AE32AF3329
:101F480074041246368F3B9000CFE0704CAE32AF2F
:101F580033900020E0FCA3E0FDEFD39DEE9C400908
:101F68001246A38E328F338006753300753200AE69
:101F780032AF33741012464490005BE08E048F0534
:101F8800FF1200858C328D337400D39D74019C4000
:101F98000585333B8003753BFF90009AE0B401024E
:101FA800800302204BA208B3B3500E90006EE0A845
:101FB80024B80005D39525500302204590006FE012
:101FC80075F019A4FFAEF09000B2E08E048F05FF03
:101FD8001200859000ABE0853BF0A4FFAEF074647E
:101FE8008D028C038E048F05FF120085EA2DFDEB10
:101FF8003CFC8C328D33E545600F9000C4E0B402A0
:10200800089000C6E0640160028017AE32AF3374F6
:10201800E7124644E5458E048F05FF1200858C3291
:102028008D33900030E0A832B8000AD395334005CC
:102038008533398006900030E0F53980069000300D
:10204800E0F5398003753B00900067E07005754C3A
:1020580002800375BB19E54CB40202800302211902
:10206800900067E07003022108E536D3940140032D
:1020780002210690001EE0FEA3E0FFE53F12469B0A
:1020880090001EEEF0A3EFF07E017F00E5BE124641
:1020980044E5BD2FFF50010E8E328F339000D4E0FF
:1020A8007013740A12464474518E048F05FF12008F
:1020B800858D3F8019AE32AF33740A1246448F04BF
:1020C8008E057E017F95CDCCCD1245468F3FE53FED
:1020D800D394644003753F6490001EE0FEA3E0FFC4
:1020E800E53F2FFF50010E90001EEEF0A3EFF09099
:1020F800006BE0048E048F05FF1200858D3F80037E
:10210800753F329000B7E07005754C03800375BBCE
:1021180013E54CB4035E9000B7E060477E017F0092
:10212800E5BE124644E5BD2FFF50010E8E328F33B7
:1021380074041246368F409000B9E08540F0A4FD43
:10214800ACF07464FF1200858D409000B8E08540C3
:10215800F0A4FFAEF074FF8E048F05FF1200858D8A
:102168004F8003754000900065E07005754C048051
:102178000375BB17E54CB40402800302221A9000D1
:1021880065E0B4017C7E017F00E5BE124644E5BDF2
:102198002FFF50010E74041246368E328F33900092
:1021A80032E06012900032E0149042EC93A832B80A
:1021B8000006953340028006900032E014F090004B
:1021C80032E0C394775013900032E0049042EC93CD
:1021D800A832B80005D3953350028006900032E04B
:1021E80004F0900032E0FE90008BE08E0088F0A4AE
:1021F800FFAEF074648E048F05FF1200858D418058
:1022080003754100900066E07005754C0580037504
:10221800BB16E54CB4050280030222AD900066E0CF
:10222800B4017C7E017F00E5BE124644E5BD2FFF68
:1022380050010E74041246368E328F33900033E00C
:102248006012900033E01490436593A832B80006FA
:10225800953340028006900033E014F0900033E09C
:10226800C394775013900033E00490436593A832E9
:10227800B80005D3953350028006900033E004F08F
:10228800900033E0FE900091E08E0088F0A4FFAE4D
:10229800F074648E048F05FF1200858D42800375EB
:1022A800420075BB1FE54CB406337E017F00E5BED6
:1022B800124644E5BD2FFF50010E8E328F3374094C
:1022C80012464474E68E048F05FF1200858D4490F3
:1022D800006DE07005754C07800375BB15E54CB4BF
:1022E800070280030223EF90006DE070030223DEF3
:1022F8007E017F00E5BE124644E5BD2FFF50010E6A
:102308008E328F3374041246368F4390006DE0B4DA
:1023180001159000C1E08543F0A4FFAEF0740712E8
:102328004636EF9007A4F090006DE0B402159000D7
:10233800C1E08543F0A4FFAEF07407124636EF9073
:1023480007A3F090006DE0B4030280030223DC9041
:1023580000AEE0701CE543C3940A5002D201E54385
:10236800D394644002C20190008DE0900059F0803F
:102378006390008DE070349000C1E08543F0A4FFC5
:10238800AEF074FF8E048F05FF120085ED900059A2
:10239800F0AE24AF25741EBE0006D39F4002D201C2
:1023A800E53BD394E54002C2018029E543C3940A82
:1023B800500DAE24AF25741EBE0004D39F5002807A
:1023C80002D201E53BD394E54002C20190008DE0C2
:1023D800900059F080037543009000C4E0700575C3
:1023E8004C08800375BB14E54CB408509000C4E059
:1023F80060397E017F00E5BE124644E5BD2FFF50DF
:10240800010E8E328F33EFD39421EE940E40057572
:1024180045FF8015AE32AF33741012464474E38E14
:10242800048F05FF1200858D4580037545009000D7
:1024380068E0600575BB1A800375BB18054CD2ECC3
:10244800AE26AF27EFD39440EE949C50030226A902
:10245800C20D7536467537467538009000A9E0708C
:1024680005754A028003754A03C293C294C291C299
:1024780092C287C290E5B554EFF5B5E5B554DFF5DE
:10248800B5C296C295C2A0C297C2A2C2A1E5B55470
:102498007FF5B5E5B554BFF5B5A21AB34008E5B563
:1024A8004404F5B58006E5B554FBF5B5A20FB35065
:1024B8000EE53BD394334007E53BC394CC4003027D
:1024C8002553E5B54401F5B57408900057F0900020
:1024D80063E075F064A4FFAEF08E348F357402BEED
:1024E800000AD39F400675350275340075A710851C
:1024F800F95185FA527E017F00E552124644E551B2
:102508002FFF50010E8E328F33AC34AD35EF2DFDD9
:10251800EE3CFC8C348D35D293D294E535F5FBE551
:1025280034F5FCE535F5E9E534F5EA9000A7E0B4C3
:102538000314D291D292E535F5EBE534F5ECE535A7
:10254800F5EDE534F5EE75A700D20FE53BC3941A17
:102558005002C20F90000874FFF0A374DCF09000E2
:102568008AE090000EF8E4F0E8A3F0C212C21474F6
:10257800C8900024F074C8900026F0C210C21175EB
:102588002500752400753D00C208756D0090001681
:10259800E4F0A3F0754D1E900799E0FEA3E0FF74E8
:1025A800031246447401124636900797EEF0A3EFE3
:1025B800F090007CE06005123DF58002C2049000B6
:1025C8007FE06005123EE58002C206A204300501E4
:1025D800B35017A204B34008E5B54408F5B5800622
:1025E800E5B554F7F5B5A2049205A206300701B384
:1025F8005017A206B34008E5B54402F5B58006E5D4
:10260800B554FDF5B5A2069207C203752B00752ACD
:1026180000900010E4F0A3F090006BE075F032A495
:10262800FFAEF090001EEEF0A3EFF090000CE4F087
:10263800A3F0C21B900058E0C3943C5019758DF06C
:10264800758B00753E15E54CB40909900058E004F7
:10265800F0754C00803BE54CB40903754C007527B8
:1026680000752600758D00758B00753E009000572B
:10267800E0C3940C5008900057E004F08006740CF6
:10268800900057F0900057E0B40C06E5B554FEF5FD
:10269800B5E544C394415009740E900034F0120219
:0426A800730209FEB2
:104274000000010001400160018001A001C001E0D3
:1042840002000300039603B603D603F404000500FA
:1042940005180530054805600578059005A805C092
:1042A400060006140628063C066E068C00FF013F35
:1042B400015F017F019F01BF01DF01FF02FF039541
:1042C40003B503D503F303FF04FF0517052F0547C3
:1042D400055F0577058F05A705BF05FF06130627AC
:1042E400063B066F068B06A9DAD8D7D5D4D2D0CF31
:1042F400CDCBC9C7C6C4C2C0BEBCBAB8B5B3B1AFD2
:10430400ADABA8A6A4A2A09D9B99969492908D8BE8
:1043140089878482807E7C79777573716F6D6B6910
:10432400676563615F5D5B5957565452504F4D4BFF
:104334004A4847454442413F3E3C3B3A393736358B
:10434400343231302F2E2D2C2B2A292827262525AF
:104354002423222121201F1E1E1D1C1C1B1A1A1976
:1043640019EEECEBEAE9E8E7E5E4E3E1E0DEDDDBC6
:10437400D9D8D6D4D2D0CECCCAC8C6C3C1BFBCBA91
:10438400B7B5B2B0ADABA8A5A3A09D9B98959290EC
:104394008D8A8785827F7D7A7775726F6D6A68658D
:1043A40063615E5C5A575553514F4D4B49474543E2
:1043B40042403E3C3B393836353332312F2E2D2B9B
:1043C4002A292827262524232221201F1E1D1D1CBF
:0A43D4001B1A1A19181817161615EF
:1026CA00750B00750A00AE0AAF0BAC08AD09EDC375
:1026DA009FEC9E401674FF12007575CF01780B743B
:1026EA000126F6500418E436F650DB2290002EE05C
:1026FA00B4AA1C90075FE0B43C1590079FE0FEA3C4
:10270A00E0FFEF4E6009741EBE0004D39F5003021F
:10271A00282475350075340075F80990079FE0FE86
:10272A00A3E0FF74076F4E6006740E6F4E70067456
:10273A003A90075FF090079FE0FEA3E0FF7408BE9F
:10274A00001ED39F401A7E017F0890079FE0FCA3DA
:10275A00E0FD1DBDFF011C1200038E328F33801F66
:10276A0090079FE0FEA3E0FF740812469B8F048E39
:10277A00057E017F08CDCCCD1200038E328F33AE99
:10278A0034AF35740CD39F74019E500302281FA2E4
:10279A00F9B3407EE5354534700375A382AE34AF94
:1027AA003574016F4E700375A300AE34AF357402F1
:1027BA006F4E700D9007A0E075F002A4FDACF08D8D
:1027CA00A3AE34AF3574036F4E700375A300AE34F5
:1027DA00AF357403BE00039F5013AC32AD33ED2FF7
:1027EA00FFEC3EFE90005B12466BE0F5A3AE34AF01
:1027FA0035EFB40B09EEB401057414120075AE344A
:10280A00AF35EFB40B07EEB4010375F80D78341247
:10281A0046AB02278990002EE4F022753500753404
:10282A000075F80990079FE0FEA3E0FF7408BE0058
:10283A001ED39F401A7E017F0890079FE0FCA3E009
:10284A00FD1DBDFF011C1200038E328F33801F90C5
:10285A00079FE0FEA3E0FF740812469B8F048E05D3
:10286A007E017F08CDCCCD1200038E328F33AE3479
:10287A00AF357411D39F74019E5003022955A2F9F2
:10288A00B35003022952E5354534700375A3D2AE1D
:10289A0034AF3574016F4E700375A300AE34AF3593
:1028AA0074026F4E700D9007A0E075F002A4FDACA3
:1028BA00F08DA3AE34AF3574036F4E700375A30069
:1028CA00AE34AF3574046F4E700375A300AE34AFE7
:1028DA003574056F4E700375A300AE34AF357406B8
:1028EA006F4E700375A300AE34AF3574076F4E7028
:1028FA000375A300AE34AF3574086F4E700375A329
:10290A0000AE34AF357408BE00039F5016AC32AD2A
:10291A0033ED2FFFEC3EFE90005612466BE5A3F016
:10292A0075A300AE34AF35EFB41009EEB4010574E7
:10293A0014120075AE34AF35EFB41007EEB40103CC
:10294A0075F80D78341246AB022878227535007571
:10295A00340075F809AE34AF357417BE0004D39F3E
:10296A005003022A2EA2F9B35003022A2BE5354559
:10297A0034700375A3D2AE34AF3574016F4E700351
:10298A0075A300AE34AF3574026F4E700D9007A078
:10299A00E075F002A4FDACF08DA3AE34AF3574033C
:1029AA006F4E700375A300AE34AF3574046F4E706A
:1029BA000375A300AE34AF3574056F4E700375A36B
:1029CA0000AE34AF3574066F4E700375A300AE3493
:1029DA00AF3574076F4E700375A300AE34AF35740C
:1029EA00086F4E700375A300AE34AF357408BE008D
:1029FA00039F500C90004012466BE5A3F075A300AC
:102A0A00AE34AF3574166F4E70057414120075AE7D
:102A1A0034AF3574166F4E700375F80D783412465C
:102A2A00AB02295F2290002EE0B4AB028003022A97
:102A3A00C975350075340075F809AE34AF357412AE
:102A4A00BE007CD39F4078A2F9B34070E535453487
:102A5A00700375A382AE34AF3574016F4E7003757F
:102A6A00A300AE34AF3574026F4E700D9007A0E02C
:102A7A0075F002A4FDACF08DA3AE34AF3574036FCC
:102A8A004E700375A300AE34AF357403BE00039FC6
:102A9A00500990004512466BE0F5A3AE34AF357489
:102AAA00116F4E70057414120075AE34AF3574117F
:102ABA006F4E700375F80D78341246AB022A442221
:102ACA00900035E4F0746490079FF8E4F0E8A3F00E
:102ADA0012295674C890079FF8E4F0E8A3F0900012
:102AEA004CE0B4371A900049E0900040F090004A58
:102AFA00E0900041F090004BE0900042F080469058
:102B0A0000357401F0746590079FF8E4F0E8A3F0CB
:102B1A0012295674C890079FF8E4F0E8A3F09000D1
:102B2A004CE0B4371A900049E0900040F090004A17
:102B3A00E0900041F090004BE0900042F080067473
:102B4A0002900035F0900036E4F0746690079FF822
:102B5A00E4F0E8A3F012295674C890079FF8E4F04D
:102B6A00E8A3F090004BE0B43712900049E09000DF
:102B7A003AF090004AE0900043F080769000367474
:102B8A0001F0746790079FF8E4F0E8A3F012295661
:102B9A0074C890079FF8E4F0E8A3F090004BE0B403
:102BAA003712900049E090003AF090004AE0900015
:102BBA0043F0803E7402900036F0746890079FF8E4
:102BCA00E4F0E8A3F012295674C890079FF8E4F0DD
:102BDA00E8A3F090004BE0B43712900049E090006F
:102BEA003AF090004AE0900043F0800674039000A7
:102BFA0036F022E55E2533FFAE3250010E90005FBB
:102C0A0012466BE0F55FE55E2533FFAE3250010EEA
:102C1A000FBF00010E90005F12466BE0F5608566FB
:102C2A0062E55FB56005855F5E8041E560D3955FCB
:102C3A00401DE560C3955F8561F0A4FFAEF0E562D3
:102C4A008E048F05FF120085ED255FF55E801DE578
:102C5A005FC395608561F0A4FFAEF0E5628E048FD4
:102C6A0005FF120085EDF404255FF55E22E560D3C9
:102C7A00955F401DE560C3955F8561F0A4FFAEF0E6
:102C8A00E5628E048F05FF120085ED255FF55E80F3
:102C9A001DE55FC395608561F0A4FFAEF0E5628E25
:102CAA00048F05FF120085EDF404255FF55E22E529
:102CBA003975F00484FF7E008F5EE53975F004846F
:102CCA00ADF07C008D61756604753201753300E5DF
:102CDA005EC3943F5005122BFD800690019EE0F5DD
:102CEA005E855E54755300900031E075F020A4FFB4
:102CFA00AEF09000B0E08E048F05FF1200858D5E65
:102D0A00900098E0D395395003022DBF9000BCE0A3
:102D1A00D395394010ED90019F124680E0F5567523
:102D2A005500022DBC900087E0D395394043E55EFB
:102D3A0090019F124680E0F55FE55E9001BF124662
:102D4A0080E0F5609000BCE0F4042539F56190005C
:102D5A0087E0FE9000BCE0F4042EF562E55FB56002
:102D6A0005855F5E8003122C77855E567555008057
:102D7A0041E55E9001BF124680E0F55FE55E900195
:102D8A00DF124680E0F560900087E0F4042539F50B
:102D9A0061900098E0FE900087E0F4042EF562E569
:102DAA005FB56005855F5E8003122C77855E567578
:102DBA005500022E669000BFE0D395395011E55EAA
:102DCA0090021F124680E0F556755500022E669055
:102DDA000088E0D395395043E55E9001FF124680A2
:102DEA00E0F55FE55E90021F124680E0F560900014
:102DFA0088E0F4042539F5619000BFE0FE90008870
:102E0A00E0F4042EF562E55FB56005855F5E800338
:102E1A00122C77855E567555008041E55E9001DF7C
:102E2A00124680E0F55FE55E9001FF124680E0F50C
:102E3A0060900098E0F4042539F561900088E0FE7E
:102E4A00900098E0F4042EF562E55FB56005855FB1
:102E5A005E8003122C77855E56755500229000D04D
:102E6A00E0F563756611753202753300AE24AF253D
:102E7A00E56375F00FA4FDACF0EDD39FEC9E402105
:102E8A00E5638E048F05FF120085ED75F010A4FF2F
:102E9A00AEF0E53975F01184FD7C00ED2FF5648004
:102EAA000EE53975F01184FF7E00EF24F0F5648594
:102EBA00645EE53975F01184AFF07E008F61122BE4
:102ECA00FD855E65AE24AF259000D0E075F00FA4B5
:102EDA00FDACF0EDD39FEC9E40287532027533109D
:102EEA0085645E122BFD85655F855E60AE24AF2525
:102EFA00E5638E048F05FF12465F8D61856362125A
:102F0A002C77855E5475530075566475550022906A
:102F1A0000D0E0F563756611753202753300AE2490
:102F2A00AF25E56375F00FA4FDACF0EDD39FEC9EE1
:102F3A004021E5638E048F05FF120085ED75F010C0
:102F4A00A4FFAEF0E53B75F01184FD7C00ED2FF592
:102F5A0064800EE53B75F01184FF7E00EF24F0F5E6
:102F6A006485645EE53B75F01184AFF07E008F6185
:102F7A00122BFD855E65AE24AF259000D0E075F07A
:102F8A000FA4FDACF0EDD39FEC9E4028753202757C
:102F9A00331085645E122BFD85655F855E60AE2405
:102FAA00AF25E5638E048F05FF12465F8D61856349
:102FBA0062122C77855E5475530090009AE0B4042F
:102FCA0053E53975F00484FF7E008F5EE53975F0AC
:102FDA000484ADF07C008D61756604753201753329
:102FEA0000E55EC3943F5005122BFD800690019EBA
:102FFA00E0F55EAE53AF54E55E12464474648E0447
:10300A008F05FF120085AE53AF54EF2DFDEE3CFC49
:10301A008C538D5475566475550022900065E0B442
:10302A000146E54175F00584FF7E008F5EE5417536
:10303A00F00584ADF07C008D617566057532057505
:10304A003300E55EC394175005122BFD80069005E8
:10305A0076E0F55EAE55AF56E55E2FFF50010E7471
:10306A006412469B8E558F56900066E0B40146E581
:10307A004275F00584FF7E008F5EE54275F0058497
:10308A00ADF07C008D61756605753205753348E5CE
:10309A005EC394175005122BFD80069005BEE0F51D
:1030AA005EAE55AF56E55E2FFF50010E74641246B0
:1030BA009B8E558F56900075E0B40249E544C3943F
:1030CA004175F00584FF7E008F5EE54475F0058446
:1030DA00ADF07C008D61756605753206753300E5C5
:1030EA005EC394135005122BFD8006900672E0F51C
:1030FA005EAE55AF56E55E2FFF50010E7464124660
:10310A009B8E558F569000B7E0B4020280030231BD
:10311A00C4E53975F01584FF7E008F5EE53975F0D8
:10312A001584ADF07C008D617566157532037533B3
:10313A00F4E55EC3940B5005122BFD800690045EE5
:10314A00E0F55EE55E75F0FFA4FFAEF09000B8E032
:10315A008E048F05FF120085ED90005AF0E5407548
:10316A00F078A4FFAEF074FF8E048F05FF1200857D
:10317A008C328D3374028C068D071246368F5EAC04
:10318A0032AD337404FF12465F8D61756604753281
:10319A000675336EE55EC3941D5005122BFD80063D
:1031AA009006EAE0F55EAE55AF56E55E2FFF500198
:1031BA000E746412469B8E558F562290006DE0B4B1
:1031CA0001179007A4E02556FFAE5550010E900056
:1031DA00C1E012469B8E558F5690006DE0B40316DF
:1031EA00A201B3B35010900059E0C39405A824B8C3
:1031FA00000695254002801090008FE02556FFAE0C
:10320A005550010E8E558F56900067E0B402028029
:10321A00030233F290006AE0602FE541D3941E4026
:10322A0028900010E0FEA3E0FF9000A5E075F003EF
:10323A00A4FDACF0EFD39DEE9C400E9000C9E0A82F
:10324A0024B80005D3952550030233F29000B2E06A
:10325A008539F0A4FFAEF07405124644740712468D
:10326A00368E328F33900071E0A824B80004952579
:10327A005012900072E075F002A4FDACF0EFC39D0D
:10328A00EE9C40030233F2E53975F00B84FF7E00B1
:10329A009005EF12466BFEE0FFEE900069E0FEEF4C
:1032AA008E0088F0A4FFAEF074648E048F05FF12BE
:1032BA0000858C328D33900031E075F018A4FFAE92
:1032CA00F09000B0E08E048F05FF1200858C068D09
:1032DA000790060712466BAE32AF33E012464474CB
:1032EA00648E048F05FF1200858C328D33E53FA86A
:1032FA0032B80077D395334072E53FC39533FFE484
:10330A009532FE8E328F337428BE00039F500C759F
:10331A003328753200740D900034F0AE32AF33901A
:10332A00006AE012464474288E048F05FF12008555
:10333A008C328D33AE53AF54740A8E048F05FF124C
:10334A0000858D068C07AC32AD33CFCECF12000389
:10335A00740A8E048F05FF1200858C328D33AE53AA
:10336A00AF541246A38E538F54807DE53FA832B8DE
:10337A00000495335072AE32AF33E53F12469B8E4E
:10338A00328F337428BE00039F500C753328753270
:10339A0000740D900034F0AE32AF3390006AE01240
:1033AA00464474288E048F05FF1200858C328D33B3
:1033BA00AE53AF54740A8E048F05FF1200858D0632
:1033CA008C07AC32AD33CFCECF120003740A8E0411
:1033DA008F05FF1200858C328D33AE53AF54EF2D1B
:1033EA00FDEE3CFC8C538D5422AE53AF54AC55AD1C
:1033FA005612000374648E048F05FF1200858C53E5
:10340A008D54900062E08C068D0712464474648ED7
:10341A00048F05FF1200858C538D54A2084017AE05
:10342A0024AF257405BE00039F5002D208E53BD3A2
:10343A0094CC4002D2029000C4E0B402089000C6C4
:10344A00E0640160028017AE53AF54E5451246446A
:10345A0074E78E048F05FF1200858C538D549000FB
:10346A0084E05402601B90007BE0A824B80012D3C9
:10347A009525400DA208B3B35007E53BC3949A4083
:10348A00028028AE5CAF5D900079E075F002A4FD81
:10349A00ACF0EF2DFDEE3CFC74022DFD50010CE565
:1034AA003BBC0007D39D4003756A01853B5D755C93
:1034BA0000E56A70030235499000D7E0C3956A4077
:1034CA0070E54175F00584FF7E0090055F12466B3A
:1034DA00E0F533753200AE32AF33900089E0124620
:1034EA004474648E048F05FF1200858C348D3590E8
:1034FA0000D7E004C3956A8C068D071246449000F3
:10350A00D7E08E048F05FF1200858C348D3590002C
:10351A007AE08C068D07124644740A8E048F05FFE2
:10352A00120085AE53AF54EF2DFDEE3CFC8C538D4B
:10353A0054056A9000D7E0C3956A5003756A0090F3
:10354A000084E05401601B900078E0A824B80012BF
:10355A00D39525400DA208B3B35007E539C394CCDF
:10356A0040028025900076E075F003A4FFAEF0E5F6
:10357A00672FFF50010E74032FFF50010EE539BE6D
:10358A000007D39F4003756B01853967E56B7003AC
:10359A000236249000D8E0C3956B4070E54175F07F
:1035AA000584FF7E0090055F12466BE0F5337532A5
:1035BA0000AE32AF33900089E012464474648E0440
:1035CA008F05FF1200858C348D359000D8E004C336
:1035DA00956B8C068D071246449000D8E08E048FB6
:1035EA0005FF1200858C348D35900077E08C068DAE
:1035FA0007124644740A8E048F05FF120085AE53E3
:10360A00AF54EF2DFDEE3CFC8C538D54056B9000AE
:10361A00D8E0C3956B5003756B00900089E0A853FE
:10362A00B8000495545009900089E0F55475530088
:10363A00229000C5E0B401028003023746A208B313
:10364A005003023744900090E0B40168AE53AF547F
:10365A00AC24AD25120003743C8E048F05FF1200C2
:10366A00859000A0E0BC00109D400D9000A2E0A84B
:10367A0053B8000495545002D203AE53AF54AC244D
:10368A00AD25120003743C8E048F05FF120085904D
:10369A0000A0E0C3940ABC0015D39D40119000A27B
:1036AA00E0C39405A853B80005D39554500280028C
:1036BA00C2038068AE53AF54AC24AD251200037424
:1036CA00788E048F05FF1200859000A0E0BC0010E0
:1036DA009D400D9000A2E0A853B8000495545004F0
:1036EA00D2038038AE53AF54AC24AD251200037414
:1036FA00788E048F05FF1200859000A0E0C3940A1B
:10370A00BC0015D39D40119000A2E0C39405A853B4
:10371A00B80005D3955450028002C203A203B340F5
:10372A0019AE53AF549000A1E012464474648E045B
:10373A008F05FF1200858C538D548002C2039000BE
:10374A00C5E0B40258E53975F00884FF7E008F5E43
:10375A00E53975F00884ADF07C008D6175660875F1
:10376A0032017533E0E55EC3943F5005122BFD80AC
:10377A000690025EE0F55EE55E75F05EA4FFAEF0CF
:10378A00740A8E048F05FF1200858C578D587402B7
:10379A00BC000AD39D4006755802755700A200B3B3
:1037AA004006A202B3B35009900016E4F0A3F080D9
:1037BA0024AE53AF547400D39F74019E400C900002
:1037CA0016E553F0A3E554F0800B74FF900016F849
:1037DA00E4F0E8A3F09000A7E0D394024006A20820
:1037EA00B3B34002800DAE53AF5474021246448EF6
:1037FA00538F54900090E0B4010DAE53AF5474024D
:10380A001246448E538F54AE53AF54745E124644DC
:10381A00740A8E048F05FF1200858C538D5474022E
:10382A00BC000AD39D4006755402755300900014DB
:10383A00E553F0A3E554F022900031E090035F12C3
:10384A004680E0F568756964900031E0FE90009B5F
:10385A00E0D39E4037E53975F00884FF7E008F5E1D
:10386A00E53975F00884ADF07C008D6175660875E0
:10387A003203753396E55EC3941F5005122BFD8003
:10388A0006900414E0F55E855E698035E53975F0C9
:10389A000884FF7E008F5EE53975F00884ADF07C00
:1038AA00008D617566087532037533B6E55EC3949B
:1038BA001F5005122BFD8006900434E0F55E855EEC
:1038CA0069229000D1E0F56375661175320475338B
:1038DA0000AE24AF25E56375F00FA4FDACF0EDD37F
:1038EA009FEC9E4021E5638E048F05FF120085ED53
:1038FA0075F010A4FFAEF0E53975F01184FD7C0077
:10390A00ED2FF564800EE53975F01184FF7E00EF26
:10391A0024F0F56485645EE53975F01184AFF07EB4
:10392A00008F61122BFD855E65AE24AF259000D114
:10393A00E075F00FA4FDACF0EDD39FEC9E40287526
:10394A00320475331085645E122BFD85655F855ED2
:10395A0060AE24AF25E5638E048F05FF12465F8DA6
:10396A0061856362122C77855E68756964229000AE
:10397A00D1E0F563756611753204753300AE24AF74
:10398A0025E56375F00FA4FDACF0EDD39FEC9E40E6
:10399A0021E5638E048F05FF120085ED75F010A4F2
:1039AA00FFAEF0E53B75F01184FD7C00ED2FF56468
:1039BA00800EE53B75F01184FF7E00EF24F0F5647C
:1039CA0085645EE53B75F01184AFF07E008F61126D
:1039DA002BFD855E65AE24AF259000D1E075F00F12
:1039EA00A4FDACF0EDD39FEC9E40287532047533EC
:1039FA001085645E122BFD85655F855E60AE24AF1F
:103A0A0025E5638E048F05FF12465F8D618563622B
:103A1A00122C77855E687569649000CCE0B40479ED
:103A2A00900031E0FE90009BE0D39E4037E5397567
:103A3A00F00884FF7E008F5EE53975F00884ADF0EA
:103A4A007C008D61756608753203753396E55EC331
:103A5A00941F5005122BFD8006900414E0F55E8534
:103A6A005E698035E53975F00884FF7E008F5EE572
:103A7A003975F00884ADF07C008D61756608753281
:103A8A00037533B6E55EC3941F5005122BFD8006FD
:103A9A00900434E0F55E855E6922900065E0B40129
:103AAA003BE54175F00584FF7E008F5EE54175F0C8
:103ABA000584ADF07C008D61756605753205753338
:103ACA0018E55EC394175005122BFD800690058EEB
:103ADA00E0F55EE569255EC39464F569900066E0E9
:103AEA00B4013BE54275F00584FF7E008F5EE54236
:103AFA0075F00584ADF07C008D617566057532053B
:103B0A00753360E55EC394175005122BFD8006904D
:103B1A0005D6E0F55EE569255EC39464F569E56856
:103B2A002569F55B90006DE0B402109007A3E025CB
:103B3A005BFE9000C1E0F4042EF55B9000C4E0D374
:103B4A0094014040E545C394E7501D74E7C3954589
:103B5A00FE9007A5E08E00F5F0E884FF7E008F5EF8
:103B6A00E55B255EF55B801CE545C394E7FE90079F
:103B7A00A5E08E00F5F0E884FF7E008F5EE55BC36A
:103B8A00955EF55BA2084006E5682464F55BE55B93
:103B9A00D394644009E55BC39464F55B8003755B69
:103BAA000090009DE0C3955B500690009DE0F55B98
:103BBA0022D2009000B3E0A824B800049525503B17
:103BCA009000B3E0A824B8000495255003755B0F54
:103BDA009000B3E004A824B8000495255003755B4F
:103BEA000A9000B3E02402A824B8000495255005E1
:103BFA00755B05C2007409900034F07E017F009065
:103C0A0000A3E01246449000B2E08E048F05FF1232
:103C1A000085E539BC000CD39D4008C200740A90A7
:103C2A000034F09000A4E0C39541500D9000B6E036
:103C3A00A824B80006952540028008C200740B909B
:103C4A000034F0A2004003755B0590006DE0B403F8
:103C5A0006A201B3B34002802B900059E0C3940539
:103C6A00A824B800049525500C90008EE0F55B74EA
:103C7A000C900034F0900059E0A824B8000495256F
:103C8A005002C200855B4690005FE0255BFE900013
:103C9A0031E075F01E84FC7F00EE2CF55B2290006B
:103CAA0031E075F00584FF7E008F5E900031E0758B
:103CBA00F00584ADF07C008D61756605753203757B
:103CCA0033D69000B0E01475F00584FF7E00E55EFF
:103CDA00BE00039F5005122BFD800BE55E90043554
:103CEA00124680E0F55EE55E9007A6F09007A6E032
:103CFA00FE90009FE0C39E500890009FE09007A6A8
:103D0A00F022E54175F00584FF7E0090055F1246BA
:103D1A006BE0F56DE56DD394644010E56DC3946472
:103D2A0075F00F84FF7E008F6D8003756D00900023
:103D3A0082E0256DF56D22900799E0FEA3E0FF74FD
:103D4A0004124636E539124644740F8E048F05FF75
:103D5A00120085900797ECF0A3EDF0900075E0B49F
:103D6A000262E544C3944175F00584FF7E008F5ECC
:103D7A00E54475F00584ADF07C008D6175660575C6
:103D8A003206753314E55EC394175005122BFD8075
:103D9A0006900686E0F55E900797E0FEA3E0FF74C2
:103DAA000A8E048F05FF120085E55E8C068D0712C8
:103DBA004644740A8E048F05FF120085900797EC1B
:103DCA00F0A3EDF0900797E0FEA3E0FF90079DE0D7
:103DDA00FCA3E0FDEDD39FEC9E400F90079DE0F819
:103DEA00A3E0900797C8F0A3C8F02290007CE0B443
:103DFA00010385255190007CE0B402129000B2E0E4
:103E0A008539F0A4FFAEF074081246368F5190003F
:103E1A007CE0B40303853B5190007CE0B404038545
:103E2A00415190007CE0B40507E542C39414F55172
:103E3A0090007CE0B4060385435190007CE0B4070F
:103E4A000385445190007CE0B408038545519000F5
:103E5A007CE0B4090385405190007DE0FE90007E2D
:103E6A00E0D39E404B90007CE0B4041890007EE0C2
:103E7A00C395515002D20490007DE0D3955140027F
:103E8A00C204802A90007DE0C39551500990007EBB
:103E9A00E0D3955150028002D20490007DE0D39580
:103EAA0051500990007EE0C395515002C204802A05
:103EBA0090007DE0D39551400990007EE0C3955172
:103ECA0040028002C20490007DE0C39551400990EF
:103EDA00007EE0D395514002D2042290007FE0B4E4
:103EEA00010385255190007FE0B402129000B2E0F0
:103EFA008539F0A4FFAEF074081246368F5190004F
:103F0A007FE0B40303853B5190007FE0B40403854E
:103F1A00415190007FE0B40507E542C39414F5517E
:103F2A0090007FE0B4060385435190007FE0B40718
:103F3A000385445190007FE0B40803854551900001
:103F4A007FE0B40903854051900080E0FE90008133
:103F5A00E0D39E4040900080E0C395515009900004
:103F6A0081E0D3955150028002D206900080E0D3BE
:103F7A0095515009900081E0C395515002C20690B4
:103F8A00007FE0B401099000BEE0D3953B50028067
:103F9A0002C206802A900080E0D395514009900021
:103FAA0081E0C3955140028002C206900080E0C3BE
:103FBA0095514009900081E0D395514002D20622E2
:103FCA00AE59AF5A74F5D39F74019E4008785912BE
:103FDA0046AB0240C5755A01755900AE24AF25E5B6
:103FEA006DBE000DD39F4009900094E0D3956E40BA
:103FFA0002801B756E00E56DC39525F551900097FB
:10400A00E0D3956C4006E56C2551F56C8002056E8F
:10401A00900070E0D3953B401CE539C3953A4015B2
:10402A00AE24AF25E56DBE00039F5009900095E0D0
:10403A00D3956F400280579007A7E0A824B80004E0
:10404A00952550037571009007A7E0A824B8000BC6
:10405A00D395254006E5259007A7F0E571702AE576
:10406A0025C3956DF551E551D39405400375510566
:10407A00900096E0C3956C5007E551C3956C4002D9
:10408A008007E56CC39551F56C756F008002056F6A
:10409A00E5717016900070E0C3953B500DE56D24F4
:1040AA0005A824B8000695254002800F900083E0F9
:1040BA00F56C75710174789007A7F022AE59AF5A62
:1040CA0074E9D39F74039E400878591246AB0242A2
:1040DA0073755A01755900756C32A21C402A756CA9
:1040EA0019900083E075F002A4FFAEF0E56EBE0001
:1040FA0006D39F4002D21C056E757103747890072F
:10410A00A7F0757000024262AE24AF25E56D6F4ECE
:10411A007003024262E56DBE000DD39F4009900014
:10412A0094E0D3956E40028017756E00A208B3B36F
:10413A005007E571C3940340028003756C19800D22
:10414A00E56DC39525F551E56E2551F56E90007024
:10415A00E0D3953B400E9007A7E0A824B80007D308
:10416A0095254002800C0570900083E0B5700375B8
:10417A007100E571B4030DE56D2402A824B80006A8
:10418A0095254002800A0570E570B43C03757102FA
:10419A00E571B402299007A7E0A824B8000ED395C8
:1041AA00254009E5259007A7F0757000900070E09A
:1041BA00C3953B500975700074789007A7F0E571B4
:1041CA00705A900070E0D3953B401CE539D3953A7C
:1041DA004015AE24AF25E56DBE00039F500990003F
:1041EA0095E0D3956F40028008756F00756C4B801F
:1041FA0028E525C3956DF551E551D394054003751E
:10420A005105900070E0D3953B4008E56F2551F5C4
:10421A006F8006E56F2406F56F757000E5717016FC
:10422A00900070E0C3953B500DE56D2405A824B8B5
:10423A000006952540028003757101E571B40118E5
:10424A00756C190570900083E0B57006757102757A
:10425A00700074789007A7F0E56C75F00AA4FFAEB9
:0A426A00F09007A1EEF0A3EFF022A0
:094680002582F582500205832217
:0F46270025E050020583258250020583F582228B
:10006400EF2F500205832582F582E5833E2EF5832A
:010074002269
:10469B00CFC39FFF50011E22C3EF9DFFEE9CFE2256
:09468900E493F608740193F62293
:0846AB000806B6000218062201
:0D465200A3E004F07006124676E004F022AA
:0E003900A3E014F0B4FF06124676E014F022A5
:0E463600048007C3CE13CECF13CFD5E0F622FB
:10454600BC000FBE0008ED8FF084FFADF022E4FE44
:10455600FF22BE000DEF60FE54F0606F20E70302FD
:1045660045FCEAC0E0EBC0E078017A0075F001EEA8
:1045760020E710EF25E0FFEE33FE0AC5F023C5F075
:1045860030E7F0EA5407F9096A7A007B006001080F
:10459600C3EC9E40167004ED9F4010ED9FFDEC9E0F
:1045A600FCE5F0CA4ACA03F5F08005E5F003F5F02C
:1045B600C3EE13FEEF13FFD9D77908CACBCAD8D0FA
:1045C600EAFEEBFFD0E0FBD0E0FA22EC8FF084FCB1
:1045D600ED54F045F0C48FF084FEEDC454F045F080
:1045E600C48FF084FDEEC4FE54F02DFFEE540F3C54
:1045F600FEADF07C0022790078008FF0EC7E08207A
:10460600E70DC3CD33CD33C933C9C833C8DEF08413
:1046160049F9E5F08FF0BE00E6FD7C00E9FFE8FE13
:014626002271
:0E464400F88FF0A4FFE5F0CE88F0A42EFE2241
:10000300EF8DF0A4F9A8F0EF8CF0A428F8EE8DF0B2
:06001300A428FEE9FF2213
:10007500600D782B02007F007830D8FED5E0F8229D
:10008500EEC0E07E00124546EFFDEEFCD0E0FE221C
:0C465F00EEC0E07E00124546D0E0FE22D6
:03001B0002001EC2
:03009B0002004917
:0300000002469223
:0946920075817275D00002038EDF
:10466B00E5822FF582E5833EF583220582D5820212
:05467B001583158222E9
:10001E00C0E0C0F0C083C082C0D075D000120339DA
:0B002E00D0D0D082D083D0F0D0E032E0
:10004900C0E0C0F0C083C082C0D075D00012033CAC
:0B005900D0D0D082D083D0F0D0E032B5
:00000001FF
